:100000000C9472000C948B000C948B000C948B005D
:100010000C948B000C948B000C948B000C948B0034
:100020000C948B000C948B000C948B000C948B0024
:100030000C948B000C948B000C948B000C948B0014
:100040000C948B000C948B000C948B000C948B0004
:100050000C948B000C948B000C948B000C948B00F4
:100060000C948B000C948B000C948B000C948B00E4
:100070000C948B000C948B000C948B000C948B00D4
:100080000C948B000C948B000C948B000C948B00C4
:100090000C948B000C948B000C948B000C948B00B4
:1000A0000C948B000C948B000C948B000C948B00A4
:1000B0000C948B000C948B000C948B000C948B0094
:1000C0000C948B000C948B000C948B000C948B0084
:1000D0000C948B000C948B000C948B000C948B0074
:1000E0000C948B0011241FBECFEFD1E2DEBFCDBF39
:1000F00000E00CBF14E0A0E0B2E0EEE7F1E000E0C9
:100100000BBF02C007900D92A03DB107D9F70E9426
:100110008D000C94BD000C940000CF93DF93CDB7FD
:10012000DEB7C05DD2400FB6F894DEBF0FBECDBFC4
:100130008FEF84B980ED92E0E0E0F2E0DE0111960D
:1001400001900D920197E1F7CE018F529D4F23E868
:1001500033E0FE0131964081329647BD24BD35BD66
:100160004FEF50E762E0415050406040E1F700C07F
:0E0170000000E817F90779F7ECCFF894FFCFFD
:10017E00800082008400860088008B008D008F0036
:10018E0091009300960098009A009C009E00A0009B
:10019E00A300A500A700A900AB00AD00AF00B10001
:1001AE00B300B500B700B900BB00BD00BF00C10071
:1001BE00C300C500C700C900CA00CC00CE00D000E5
:1001CE00D100D300D500D600D800DA00DB00DD0068
:1001DE00DE00E000E100E300E400E500E700E800F7
:1001EE00E900EA00EC00ED00EE00EF00F000F10097
:1001FE00F200F300F400F500F600F700F700F80047
:10020E00F900F900FA00FB00FB00FC00FC00FD0009
:10021E00FD00FD00FE00FE00FE00FF00FF00FF00DF
:10022E00FF00FF00FF00FF00FF00FF00FF00FF00C8
:10023E00FE00FE00FE00FD00FD00FD00FC00FC00C7
:10024E00FB00FB00FA00F900F900F800F700F700D8
:10025E00F600F500F400F300F200F100F000EF00FC
:10026E00EE00ED00EC00EA00E900E800E700E50032
:10027E00E400E300E100E000DE00DD00DB00DA0078
:10028E00D800D600D500D300D100D000CE00CC00CF
:10029E00CA00C900C700C500C300C100BF00BD0031
:1002AE00BB00B900B700B500B300B100AF00AD00A0
:1002BE00AB00A900A700A500A300A0009E009C0013
:1002CE009A0098009600930091008F008D008B008D
:1002DE00880086008400820080007D007B0079000B
:1002EE0077007400720070006E006C006900670089
:1002FE006500630061005F005C005A005800560004
:10030E005400520050004E004C004A004800460077
:10031E004400420040003E003C003A0038003600E7
:10032E003500330031002F002E002C002A0029004A
:10033E00270025002400220021001F001E001C00A3
:10034E001B001A00180017001600150013001200EB
:10035E00110010000F000E000D000C000B000A0023
:10036E00090008000800070006000600050004004A
:10037E00040003000300020002000200010001005D
:10038E00010000000000000000000000000000005E
:10039E00000000000000000001000100010002004A
:1003AE000200020003000300040004000500060022
:1003BE00060007000800080009000A000B000C00E8
:1003CE000D000E000F00100011001200130015009A
:1003DE001600170018001A001B001C001E001F003C
:1003EE002100220024002500270029002A002C00CD
:1003FE002E002F00310033003500360038003A0051
:10040E003C003E00400042004400460048004A00C6
:10041E004C004E00500052005400560058005A0036
:10042E005C005F00610063006500670069006C009E
:10043E006E00700072007400770079007B007D0002
:00000001FF
